:100000000C945D000C9485000C9485000C94850084
:100010000C9485000C9485000C9485000C9485004C
:100020000C9485000C9485000C9485000C9485003C
:100030000C9485000C9485000C9485000C9485002C
:100040000C940E010C9485000C947E010C945801C4
:100050000C9485000C9485000C9485000C9485000C
:100060000C9485000C94850000000008000201003B
:100070000003040700000000000000000000000072
:10008000250028002B0000000000240027002A0083
:10009000040404040404040402020202020203032E
:1000A0000303030301020408102040800102040836
:1000B0001020010204081020F32111241FBECFEFED
:1000C000D8E0DEBFCDBF12E0A0E0B1E0ECEAFCE496
:1000D00002C005900D92AA37B107D9F723E0AAE72D
:1000E000B2E001C01D92A333B207E1F710E0CDE505
:1000F000D0E004C02197FE010E942125CC35D10714
:10010000C9F70E94AF1D0C9454260C940000CF92A6
:10011000DF92EF92FF920F931F93CF93DF936C01C7
:100120007A018B01C0E0D0E0CE15DF0581F0D80167
:100130006D918D01D601ED91FC910190F081E02D42
:10014000C6010995892B11F02196EECF7E01C701DA
:10015000DF91CF911F910F91FF90EF90DF90CF90A3
:100160000895089580E090E008950E9448268CE864
:1001700092E00E94E10121E0892B09F420E0822F26
:100180000895EF92FF920F931F93CF93DF93EC01AB
:1001900081E0888F9B8D8C8D981305C0E889F98943
:1001A000808185FD26C0F62E0B8D10E00F5F1F4F5E
:1001B0000F731127E02E8C8DE8120CC00FB607FCD0
:1001C000FACFE889F989808185FFF5CFCE010E94B9
:1001D0006F07F1CF8B8DFE01E80FF11DE35AFF4F42
:1001E000F0829FB7F8940B8FEA89FB898081806247
:1001F0000AC09FB7F894EE89FF896083E889F9897E
:1002000080818370806480839FBF81E090E0DF9174
:10021000CF911F910F91FF90EF9008951F920F9231
:100220000FB60F9211242F933F938F939F93AF9309
:10023000BF938091800290918102A0918202B0913F
:10024000830230917F0223E0230F2D3720F40196A3
:10025000A11DB11D05C026E8230F0296A11DB11DE9
:1002600020937F028093800290938102A093820268
:10027000B09383028091850290918602A0918702BB
:10028000B09188020196A11DB11D809385029093C3
:100290008602A0938702B0938802BF91AF919F918D
:1002A0008F913F912F910F900FBE0F901F90189537
:1002B0001F920F920FB60F9211242F933F934F93DB
:1002C0005F936F937F938F939F93AF93BF93EF93BE
:1002D000FF938CE892E00E946F07FF91EF91BF912E
:1002E000AF919F918F917F916F915F914F913F91CE
:1002F0002F910F900FBE0F901F9018951F920F9285
:100300000FB60F9211242F938F939F93EF93FF9328
:10031000E0919C02F0919D028081E091A202F09117
:10032000A30282FD12C090818091A5028F5F8F731E
:100330002091A602821751F0E091A502F0E0E45767
:10034000FD4F958F8093A50201C08081FF91EF91B1
:100350009F918F912F910F900FBE0F901F90189526
:10036000FC01538D448D252F30E0842F90E0821BBB
:10037000930B541710F0CF96089501970895FC0140
:10038000918D828D981761F0828DDF01A80FB11DCC
:100390005D968C91928D9F5F9F73928F90E00895F0
:1003A0008FEF9FEF0895FC01918D828D981731F0AA
:1003B000828DE80FF11D858D90E008958FEF9FEFFE
:1003C0000895FC01918D228D892F90E0805C9F4FD4
:1003D000821B91098F739927089580E090E0892B03
:1003E00029F00E94B70081110C9400000895DC01EF
:1003F000ED91FC910484F585E02D6DE070E00994A9
:10040000FC0197859F7121F490899F7781E009F025
:1004100080E00895FC0197859F719D3029F49089B3
:100420009F7781E0903509F080E008959B0177FF88
:1004300002C0295F3F4F43E0359527954A95E1F784
:10044000FC01E20FF31F278530E0CB0168E070E08C
:100450000E94F924A90102C0559547958A95E2F7B3
:10046000CA0181700895660F771F860F971FFC01E0
:10047000828980580895660F771F860F971FFC01A9
:10048000818980580895860F971FFC0181890895FE
:10049000FC0114A60895FC0184A50895860F971FFA
:1004A0004195FC0141870895860F971FFC01418704
:1004B00008959B014423E9F077FF02C0295F3F4F75
:1004C00053E0359527955A95E1F7FC01E20FF31FAC
:1004D000CB0168E070E00E94F92421E030E0A9013E
:1004E00002C0440F551F8A95E2F7CA019381892BF8
:1004F0001DC077FF02C0295F3F4F43E03595279528
:100500004A95E1F7FC01E20FF31FCB0168E070E0D0
:100510000E94F92421E030E0A90102C0440F551FD8
:100520008A95E2F7CA018095938189238383089590
:10053000660F771FFC01E60FF71F8FE7489F402DDE
:1005400011244058468308956F5F7F4F660F771FD1
:10055000FC01E60FF71F8FE7489F402D11244058FC
:1005600043830895660F771F860F971F4058FC013D
:10057000468308956F5F7F4F660F771F860F971F23
:100580004058FC0143830895FC01138280E8848372
:100590008583868387838087118612860895CF920C
:1005A000DF92EF92FF920F931F93CF93DF938C0113
:1005B000EB017A01DC0115968D919C9116978130A3
:1005C000910521F0029709F45DC014C0E881F9811A
:1005D0000288F389E02DCB010995882331F082E070
:1005E00090E0F80196838583C3C1D80116961C92CA
:1005F0001E921597D701ED91FC91C284D384E881B6
:10060000F9810084F185E02D60E070E0CE0109956C
:10061000682F880F770B880B990B0E94D723AB01AB
:10062000BC01C8010E94460D482F60E070E0C70180
:10063000F6010995D701ED91FC91C484D584E88138
:10064000F9810284F385E02D60E070E0CE01099528
:10065000682F880F770B880B990B0E94D723AB016B
:10066000BC01C8010E94460D482F60E070E0C70140
:10067000F601DF91CF911F910F91FF90EF90DF90E6
:10068000CF900994D8011396ED91FC91149734966C
:10069000EE0FFF1FE00FF11F4081518157FF02C095
:1006A0004F5F5F4F55954795D701ED91FC910284BF
:1006B000F385E02D60E070E0C7010995D80113963D
:1006C000ED91FC9114973896EE0FFF1FE00FF11F8C
:1006D0004081518157FF02C04F5F5F4F559547954D
:1006E000D701ED91FC910484F585E02D60E070E088
:1006F000C7010995E881F9810288F389E02DCE01CF
:100700000995882309F44DC1F8018781E881F981B1
:100710000484F585E02D882309F461C062E070E06F
:10072000CE010995811174C1E881F9810484F585B0
:10073000E02D63E070E0CE010995811169C1E88187
:10074000F9810484F585E02D61E070E0CE01099522
:1007500081115EC1E881F9810484F585E02D60E0B6
:1007600070E0CE010995811153C1E881F9810484BB
:10077000F585E02D68E070E0CE010995811148C152
:10078000E881F9810484F585E02D69E070E0CE010F
:10079000099581113DC1E881F9810484F585E02D39
:1007A0006AE070E0CE010995811132C1E881F981DA
:1007B0000484F585E02D6BE070E0CE010995811190
:1007C00027C1E881F9810484F585E02D64E070E0BB
:1007D000CE01099581111CC1F801178219C163E08E
:1007E00070E0CE0109958823C1F0D8011396ED91F0
:1007F000FC911497EE0FFF1FE00FF11F808591858C
:100800008230910514F0019702C081E090E0918759
:10081000808781E0F8018783FBC0E881F981048447
:10082000F585E02D62E070E0CE0109958823A1F006
:10083000D8011396ED91FC911497EE0FFF1FE00F76
:10084000F11F208531858089918901972817390703
:10085000F4F6C9010196DBCFE881F9810484F585BE
:10086000E02D61E070E0CE0109958823A1F0D80168
:100870001396ED91FC911497EE0FFF1FE00FF11FFF
:10088000208931898085918501968217930704F527
:10089000C90101971DC0E881F9810484F585E02D27
:1008A00060E070E0CE0109958823A9F0D801139685
:1008B000ED91FC911497EE0FFF1FE00FF11F80895F
:1008C00091898F3F910514F4019602C08FEF90E05B
:1008D000918B808B9ECFE881F9810484F585E02D92
:1008E00064E070E0CE010995882381F0D801139669
:1008F000ED91FC911497EE0FFF1FE00FF11F118691
:1009000010868FE790E0918B808B47C0E881F9815A
:100910000484F585E02D6BE070E0CE010995882315
:1009200021F0F8011482138223C0E881F981048444
:10093000F585E02D68E070E0CE010995882341F04F
:1009400081E090E0D80114969C938E93139726C073
:10095000E881F9810484F585E02D6AE070E0CE013C
:100960000995882339F082E090E0F801948383832D
:1009700081E051CFE881F9810484F585E02D69E0BB
:1009800070E0CE010995882309F442C083E090E02D
:10099000D80114969C938E93139781E017968C93AD
:1009A00037C08091290390912A03892B61F1780146
:1009B000B8E0EB0EF11CC0E0D0E0F7016081F2E09E
:1009C000EF0EF11C8091290390912A038C0F9D1F3B
:1009D0000E9496148091290390912A038C0F9D1FE9
:1009E000D70116966C9101960E9496142296C830F3
:1009F000D10519F78091290390912A03F8016381A9
:100A000008960E949614D80116961C921E9215976D
:100A1000DF91CF911F910F91FF90EF90DF90CF90DA
:100A200008956F927F928F929F92AF92BF92CF92D2
:100A3000DF92EF92FF920F931F93CF93DF9300D03B
:100A400000D0CDB7DEB78C01DC0191968C919197E7
:100A50008111E1C088E0E3EBF1E01F9601900D9277
:100A60008A95E1F7D801AE58BF4F80E090E067E08B
:100A700070E041E050E09C0127703327FB01E21B4E
:100A8000F30B3A0102C0660C771CEA95E2F793017A
:100A9000FC0133E0F595E7953A95E1F7E00FF11F9A
:100AA000378523232D9301968034910521F7780112
:100AB00062E2E60EF11C80E4D7011D928A95E9F707
:100AC0001C8261E0CE0104960E94560C6AE070E040
:100AD000C7010E94010DC8018E549F4F2AE0FC01FE
:100AE00011922A95E9F74701F70140E050E077E0DD
:100AF000C72ED12CA1919A0163E0359527956A956F
:100B0000E1F7200F311F590162EBA60EB11C61E025
:100B100070E0A11102C060E070E0DA01A770BB27AD
:100B200036016A1A7B0A01C0660F6A94EAF7D90196
:100B3000AE54BF4F2C91622BD5016C934F5F5F4F2A
:100B400040355105B9F6FC01208121110AC0F80198
:100B5000ED54FF4F2081211104C0319620812223C2
:100B600029F081E0D80191968C9306C04AE050E0CC
:100B700062E071E00E944D268AE0EFE4F1E0D801E6
:100B8000579601900D928A95E1F780E5F701119251
:100B90008A95E9F781E4898361E0CE0101960E949C
:100BA000560C6AE070E0C7010E94010D019779F5CB
:100BB0008AE0F8017796DF011D928A95E9F720E037
:100BC00030E047E050E0F40161914F01F90193E01A
:100BD000F595E7959A95E1F7E00FF11F81E090E038
:100BE000611102C080E090E0B901677077273A0197
:100BF000661A770A01C0880F6A94EAF79789892BE9
:100C0000878B2F5F3F4F20353105E9F6B8C0D801FB
:100C100091961C92B4C0D8011896ED91FC91199749
:100C20008281811103C0ECE0F1E002C0EFE0F1E06D
:100C300080819181A28189839A83AB8363E0CE0115
:100C400001960E94560C7801B2E2EB0EF11C68E0AE
:100C500070E0C7010E94010DF80182A5882309F404
:100C60008CC020E4F701C8018E589F4FDC01019031
:100C70000D922A95E1F728E0F8013F96DF011D92D9
:100C80002A95E9F7DC0120E030E047E050E06D9183
:100C9000F90183E0F595E7958A95E1F7E00FF11FFB
:100CA00081E090E0611102C080E090E0B9016770DE
:100CB00077273A01661A770A01C0880F6A94EAF723
:100CC0009785892B87872F5F3F4F20343105F9F6B1
:100CD00061E571E0F80120E030E0DB015D91BD01EC
:100CE000818990E0418D450F841B910947FD9395C3
:100CF00097FD07C08F3F910529F024F08FEF90E01A
:100D000001C080E0818BA8014E575F4F982F9078EB
:100D1000DA019C934F5F5F4F982F9074DA019C9398
:100D20004F5F5F4F982F9072DA019C934F5F5F4F38
:100D3000982F9071DA019C934F5F5F4F982F9870B6
:100D4000DA019C934F5F5F4F982F9470DA019C9368
:100D50004F5F5F4F982F9270DA019C934F5F5F4F08
:100D60008170DA018C932F5F3F4F3196085F1F4FE0
:100D70002630310509F0B1CF02C0F80111A20F9061
:100D80000F900F900F90DF91CF911F910F91FF90D7
:100D9000EF90DF90CF90BF90AF909F908F907F901B
:100DA0006F9008950C94BF2560E070E00C94CE0B1A
:100DB000EF92FF920F931F93CF93DF93CDB7DEB7E0
:100DC00028970FB6F894DEBF0FBECDBF8C01FC0193
:100DD000E85BFE4F8081833440F4813408F057C0D3
:100DE000882331F08034E9F06DC08F3F09F06AC08C
:100DF00089E0F8018383148283E0858380E8868319
:100E00001782108611861286FF24F394F386F486E7
:100E100040E063E0C80103960E94190BF801F4A6B4
:100E20004CC08091840298012C5D3F4F7901811163
:100E30000CC028E0C8010396FC01D70101900D9277
:100E40002A95E1F741E068E00CC088E0F901DE0195
:100E5000119601900D928A95E1F741E068E0CE018C
:100E600001960E94190BF801EF2811F4128207C0B5
:100E7000E65BFE4F808181708083F801828361E0B0
:100E800070E0C8010E94CE0B809384021BC0F80161
:100E9000138280E884838583868387838087118695
:100EA000128682E08387848741E06AE0C801039666
:100EB0000E94190B81E0F80184A761E070E0C8018D
:100EC0000E94CE0B28960FB6F894DEBF0FBECDBFA2
:100ED000DF91CF911F910F91FF90EF900895FC014A
:100EE000848DDF01A80FB11DA35ABF4F2C91848DB3
:100EF00090E001968F739927848FA689B7892C93E8
:100F0000A089B1898C91837080648C93938D848D3A
:100F1000981306C00288F389E02D80818F7D80833D
:100F20000895CF93DF93EC01888D8823C9F0EA8977
:100F3000FB89808185FD05C0A889B9898C9186FDD2
:100F40000FC00FB607FCF5CF808185FFF2CFA889CF
:100F5000B9898C9185FFEDCFCE010E946F07E7CF55
:100F6000DF91CF910895CF92DF92EF92FF920F938E
:100F70001F93CF93DF93EC011A828FEB91E099835B
:100F800088831C821B82198618868FE790E0998BD4
:100F9000888B1B861A869B8B8A8B1D861C869D8B55
:100FA0008C8B1F861E869F8B8E8B00912903109140
:100FB0002A030115110509F05DC082E00E94F708BF
:100FC0008C0190932A0380932903009779F569E0B7
:100FD00070E082E00E946C0890932A0380932903BA
:100FE000892B09F46BC000E010E0809129039091F7
:100FF0002A0360E0800F911F0E94961480912903BC
:1010000090912A03800F911F6FE701960E9496141A
:101010000E5F1F4F0830110541F780912903909111
:101020002A0360E008960E94961448C008960E9421
:10103000A52290E09C838B837E0188E0E80EF11C62
:101040006E01E0E1CE0ED11CC8010E94A52290E005
:10105000F701819391937F01C80101960E94A52217
:1010600090E0F701978386830E5F1F4FCE14DF0455
:1010700059F724C0C80108960E94A52290E09C83DD
:101080008B837E01F8E0EF0EF11C6E0180E1C80E4B
:10109000D11CC8010E94A52290E0F7018193919391
:1010A0007F01C80101960E94A52290E0F701978375
:1010B00086830E5F1F4FEC14FD0459F781E090E02A
:1010C0009E838D83DF91CF911F910F91FF90EF90C1
:1010D000DF90CF90089508958F929F92AF92BF9224
:1010E000CF92DF92EF92FF920F931F93CF93DF93F4
:1010F000C82E5B01E0908A02F0908B02C0E0D0E045
:101100000AE010E0EC16FD060CF462C0C8010E9473
:10111000A52298012E5F3F4F49018F3F21F0EC1629
:10112000FD0609F04CC0C4010E94A522D82EEC1681
:10113000FD0651F090E08A159B050CF440C09C2FF1
:101140008D2FE701E92EF82E6C2DC8010E94961410
:1011500060E0C80101960E9496140D5F1F4FEC16C7
:10116000FD06A1F08D2D90E00297A816B9068CF42B
:101170007801EA0CFB1C6FEFC7010E9496146D2DDD
:101180006A196350C70102960E94961421966A2D2F
:1011900001C06D2DC4010E94961480918A02909125
:1011A0008B028C179D0749F0D0938B02C0938A0263
:1011B0006C2F81E090E00E949614C8010BC0C4011E
:1011C0000E94A52290E00396080F191F21969ACF3E
:1011D00080E090E0DF91CF911F910F91FF90EF9011
:1011E000DF90CF90BF90AF909F908F900895DF9247
:1011F000EF92FF920F931F93CF93DF93D82EE0903F
:101200008A02F0908B0200E010E0CAE0D0E00E15F8
:101210001F05CCF4CE010E94A522D81209C0CE0130
:1012200001960E94A522811103C0CE0103960DC034
:10123000CE0102960E94A52290E00396C80FD91F06
:101240000F5F1F4FE4CF80E090E0DF91CF911F91BF
:101250000F91FF90EF90DF9008950F931F93CF931E
:10126000DF93EC018B018E819F81009721F00E941A
:10127000BF251F821E828A819B81009711F00E94E8
:10128000BF251B830A83DF91CF911F910F91089592
:101290000F931F93CF93DF93EC018B018C819D8182
:1012A000009711F00E94BF251D830C83DF91CF9121
:1012B0001F910F9108950F931F93CF93DF93EC012C
:1012C000142F022F6230F9F0633069F1613069F058
:1012D00085E090E00E942725FC011282D483C3831D
:1012E0008DED91E0918380832EC086E090E00E9496
:1012F0002725FC011283D483C38385ED91E091837C
:101300008083158220C087E090E00E942725FC01A1
:101310001283D483C38385EC91E09183808381E041
:10132000011110C00EC087E090E00E942725FC014B
:101330001283D483C3838DEC91E09183808381E019
:10134000011180E08683CF01DF91CF911F910F9132
:1013500008952F923F924F925F926F927F928F9259
:101360009F92AF92BF92CF92DF92EF92FF920F9334
:101370001F93CF93DF93CDB7DEB728970FB6F894BE
:10138000DEBF0FBECDBF9E838D836A017B0120E04F
:1013900030E040E053E4C701B6010E9487241816EC
:1013A00054F420E030E040E853E4C701B6010E9465
:1013B000BB226B017C0120E030E0A901C701B6012E
:1013C0000E94282387FF0BC0F7FAF094F7F8F094F7
:1013D000812C912C90E8A92E9FEBB92E13C020E010
:1013E00030E0A901C701B6010E942823882339F003
:1013F000812C912C80E8A82E8FE3B82E03C0812C7D
:10140000912C5401ED81FE8127803084B101032CA1
:10141000000C880B990B0E94D7232B013C01A701DC
:1014200096010E942823ED81FE8118160CF4B5C0A8
:1014300001851285B801012E000C880B990B0E94C2
:10144000D72369837A838B839C83A70196010E94AB
:10145000872418160CF041C0ED81FE810584F685C5
:10146000E02DFA83E983ED81FE816385748529810E
:101470003A81621B730B072E000C880B990B0E949C
:10148000D7236D837E838F839887A3019201C70141
:10149000B6010E94BB229B01AC016D817E818F81D0
:1014A00098850E948C246B017C01B8016219730934
:1014B000072E000C880B990B0E94D7239B01AC01CF
:1014C000C701B6010E942D236B017C01E981FA81DD
:1014D000BF01FF0F880B990B40C020E030E04EEFBA
:1014E00052E4C701B6010E94282387FF3DC0ED8169
:1014F000FE81238434846FE770E062197309072E3C
:10150000000C880B990B0E94D7232B013C012981E9
:101510003A814B815C81C701B6010E94BB229B01CD
:10152000AC01C301B2010E948C246B017C012FE746
:1015300030E0201B310BB901330F880B990B0E944F
:10154000D7239B01AC01C701B6010E942D236B017B
:101550007C01B101330C880B990B0E94D7239B01AE
:10156000AC01C701B60116C020E030E04EEF52E4F6
:10157000C701B6010E94BB2220E030E0A9010E9411
:101580008C2420E030E0A9010E942D2320E030E0EF
:101590004EEF52E40E94BC2210C065857685072E6E
:1015A000000C880B990B0E94D723A70196010E947B
:1015B0008C24A30192010E942D23A50194010E9475
:1015C0008C246B017C0120E030E040E053EC0E9471
:1015D000282387FD10C020E030E04EEF52E4C70121
:1015E000B6010E94872418164CF0C701B6010E946C
:1015F0009F23CB0105C080E89FEF02C08FE790E0FA
:1016000028960FB6F894DEBF0FBECDBFDF91CF9105
:101610001F910F91FF90EF90DF90CF90BF90AF9010
:101620009F908F907F906F905F904F903F902F9002
:101630000895FC0128E0539A808190E0880F892F5B
:10164000881F990B892B09F430C0000000000000AE
:10165000000000000000000000005398000000009F
:10166000000000000000000000000000000000007A
:10167000000000000000000000000000000000006A
:10168000000000000000000000000000000000005A
:10169000000000000000000000000000000000004A
:1016A000000000000000000030C00000000000004A
:1016B000000000000000000000000000000000002A
:1016C000000000000000000000000000000000001A
:1016D000000000000000000000000000000000000A
:1016E00000000000000000000000000000000000FA
:1016F00000000000000000000000000000000000EA
:1017000000000000000000005398215069F0000024
:1017100000000000000000000000000000000000C9
:101720008081880F808387CF0000000000000000C8
:10173000615031F0000000000000000031967ACFC7
:101740000000000000000000000000000000000099
:10175000539A00000000000000000000000000009C
:101760000000000000000000000000000000000079
:10177000442391F000000000000000000000000081
:101780000000000000000000000000000000000059
:10179000000000000000000053980895CF93DF93ED
:1017A000DC01FC01E85BFE4F83E0EF0119928A95B2
:1017B000E9F7EF01161617069CF484EC99E04B99B3
:1017C00007C081E09C968C939C9728E030E01BC07A
:1017D0000197A9F79C968C919C97882309F461C086
:1017E0009C968C919C9781110AC080E290E04B9965
:1017F00002C080E290E0019718161906C4F328E0B1
:1018000030E04B99FECF0000000000000000000017
:1018100000000000000000000000000000000000C8
:1018200000000000000000000000000000000000B8
:1018300000000000000000000000000000000000A8
:101840000000000000000000000000000000000098
:1018500000004B9B03C0808181608083215031094F
:1018600031F08081880F80834B9BFECFCACF888167
:10187000803441F4CD01865B9E4FE817F90711F0E3
:101880003196BDCF4B9BFECF8CE090E04B9902C0D0
:101890008CE090E0019718161906C4F381E090E0FF
:1018A00002C080E090E0DF91CF910895FC0128E034
:1018B0008AB180638AB9808190E0880F892F881F60
:1018C000990B892B09F432C00000000000000000D1
:1018D00000000000000000008AB18F7C8AB900007F
:1018E00000000000000000000000000000000000F8
:1018F00000000000000000000000000000000000E8
:1019000000000000000000000000000000000000D7
:1019100000000000000000000000000000000000C7
:101920000000000000000000000032C000000000C5
:1019300000000000000000000000000000000000A7
:101940000000000000000000000000000000000097
:101950000000000000000000000000000000000087
:101960000000000000000000000000000000000077
:101970000000000000000000000000000000000067
:10198000000000000000000000008AB18F7C8AB9CE
:10199000215069F00000000000000000000000007D
:1019A0000000000000008081880F808381CF00004C
:1019B000000000000000615031F000000000000055
:1019C0000000319674CF000000000000000000000D
:1019D0000000000000008AB180638AB900000000A6
:1019E00000000000000000000000000000000000F7
:1019F000000000000000000000008AB18F7C8AB95E
:101A00000895FC01660F660F660F9FE329B12073EE
:101A100029F09150D9F780E090E00895000000008F
:101A200000000000000000000000000000000000B6
:101A300000000000000000000000000000000000A6
:101A40000000000000000000000000000000000096
:101A50000000000000000000000000000000000086
:101A6000000000000000000099B190739193615054
:101A700051F09FE329B1207309F0C7CF9150D1F7FE
:101A800082E090E0089581E090E008954F925F92A7
:101A90006F927F928F929F92AF92BF92CF92DF927E
:101AA000EF92FF92CF93DF93EC016A017B0120E07C
:101AB00030E040E053E4C701B6010E9487241816C5
:101AC00054F420E030E040E853E4C701B6010E943E
:101AD000BB226B017C0120E030E0A901C701B60107
:101AE0000E94282387FF0BC0F7FAF094F7F8F094D0
:101AF000812C912C40E8A42E4FEBB42E13C020E093
:101B000030E0A901C701B6010E942823882339F0DB
:101B1000812C912C30E8A32E3FE3B32E03C0812CFF
:101B2000912C54018B819C81880F991FC80FD91F5C
:101B300068857985072E000C880B990B0E94D723A6
:101B40002B013C01A70196010E94872487FF44C016
:101B5000A3019201C701B6010E94BB226B017C0167
:101B6000A301920160E070E08EEF92E40E94BB223C
:101B70009B01AC01C701B6010E942D236B017C01C2
:101B800068897989072E000C880B990B0E94D7234E
:101B90009B01AC01C701B6010E948C24A5019401F0
:101BA0000E948C246B017C0120E030E040E053EC8B
:101BB0000E94282387FD13C020E030E04EEF52E45E
:101BC000C701B6010E948724181664F0C701B60148
:101BD0000E949F23CB0108C080E090E005C080E810
:101BE0009FEF02C08FE790E0DF91CF91FF90EF90E1
:101BF000DF90CF90BF90AF909F908F907F906F902D
:101C00005F904F900895CF93DF9390E0FC01EC55E7
:101C1000FF4F2491FC01E057FF4F84918823C1F0CE
:101C200090E0880F991FFC01EA57FF4FC591D491AE
:101C3000FC01E458FF4FA591B4919FB7F8948881B7
:101C4000E22FE0958E2388838C91E823EC939FBF4D
:101C5000DF91CF91089590E0FC01E859FF4F249166
:101C6000FC01EC55FF4F3491FC01E057FF4FE4912C
:101C7000EE23B9F1222339F1233091F038F42130E9
:101C8000A9F0223001F584B58F7D12C0273091F084
:101C90002830A1F02430B9F4809180008F7D03C0FA
:101CA000809180008F77809380000DC084B58F77FE
:101CB00084BD09C08091B0008F7703C08091B000CF
:101CC0008F7D8093B000F0E0EE0FFF1FE458FF4FD0
:101CD000A591B4919FB7F8948C91309538233C939B
:101CE0009FBF0895682F8CE892E00C94C1003FB725
:101CF000F8948091850290918602A0918702B0911C
:101D0000880226B5A89B05C02F3F19F00196A11D9A
:101D1000B11D3FBFBA2FA92F982F8827820F911D81
:101D2000A11DB11DBC01CD0142E0660F771F881FC8
:101D3000991F4A95D1F70895EF92FF920F931F9341
:101D4000CF93DF938B01EA01E881F981E284F38488
:101D5000DB01ED91FC910084F185E02D61E070E004
:101D6000C8010995482F61E070E0CE01F70109959F
:101D7000E881F981E484F584D801ED91FC91028435
:101D8000F385E02D61E070E0C8010995482F61E01E
:101D900070E0CE01F7010995E881F981E284F384CE
:101DA000D801ED91FC910084F185E02D62E070E0B6
:101DB000C8010995482F62E070E0CE01F70109954E
:101DC000E881F981E484F584D801ED91FC910284E5
:101DD000F385E02D62E070E0C8010995482F62E0CC
:101DE00070E0CE01F7010995E881F981E688F7886E
:101DF000D801ED91FC910484F585E02D64E070E05C
:101E0000C8010995482F64E070E0CE01F7010995FB
:101E1000E881F981E688F788D801ED91FC91048486
:101E2000F585E02D6CE070E0C8010995482F6CE065
:101E300070E0CE01F7010995E881F981E688F7881D
:101E4000D801ED91FC910484F585E02D63E070E00C
:101E5000C8010995482F61E070E0CE01F7010995AE
:101E6000E881F981E688F788D801ED91FC91048436
:101E7000F585E02D61E070E0C8010995482F62E02A
:101E800070E0CE01F7010995E881F981E688F788CD
:101E9000D801ED91FC910484F585E02D62E070E0BD
:101EA000C8010995482F63E070E0CE01F70109955C
:101EB000E881F981E688F788D801ED91FC910484E6
:101EC000F585E02D60E070E0C8010995482F60E0DD
:101ED00070E0CE01F7010995E881F981E688F7887D
:101EE000D801ED91FC910484F585E02D6DE070E062
:101EF000C8010995482F6DE070E0CE01F701099502
:101F0000E881F981E688F788D801ED91FC91048495
:101F1000F585E02D6EE070E0C8010995482F6EE070
:101F200070E0CE01F7010995E881F981E688F7882C
:101F3000D801ED91FC910484F585E02D6BE070E013
:101F4000C8010995482F6BE070E0CE01F7010995B3
:101F5000E881F981E688F788D801ED91FC91048445
:101F6000F585E02D6AE070E0C8010995482F6AE028
:101F700070E0CE01F7010995E881F981E688F788DC
:101F8000D801ED91FC910484F585E02D68E070E0C6
:101F9000C8010995482F68E070E0CE01F701099566
:101FA000E881F981E688F788D801ED91FC910484F5
:101FB000F585E02D69E070E0C8010995482F69E0DA
:101FC00070E0CE01F701DF91CF911F910F91FF904B
:101FD000EF900994EF92FF920F931F93CF93DF93AB
:101FE0008B01EA01E881F981E284F384DB01ED9160
:101FF000FC910084F185E02D61E070E0C801099555
:10200000482F61E070E0CE01F7010995E881F98180
:10201000E484F584D801ED91FC910284F385E02DF0
:1020200061E070E0C8010995482F61E070E0CE01E1
:10203000F7010995E881F981E284F384D801ED91F3
:10204000FC910084F185E02D62E070E0C801099503
:10205000482F62E070E0CE01F7010995E881F9812F
:10206000E484F584D801ED91FC910284F385E02DA0
:1020700062E070E0C8010995482F62E070E0CE018F
:10208000F7010995E881F981E688F788D801ED9193
:10209000FC910484F585E02D64E070E0C8010995A9
:1020A000482F64E070E0CE01F7010995E881F981DD
:1020B000E688F788D801ED91FC910484F585E02D40
:1020C0006CE070E0C8010995482F6CE070E0CE012B
:1020D000F7010995E881F981E688F788D801ED9143
:1020E000FC910484F585E02D60E070E0C80109955D
:1020F000482F61E070E0CE01F7010995E881F98190
:10210000E688F788D801ED91FC910484F585E02DEF
:1021100063E070E0C8010995482F62E070E0CE01ED
:10212000F7010995E881F981E688F788D801ED91F2
:10213000FC910484F585E02D61E070E0C80109950B
:10214000482F63E070E0CE01F7010995E881F9813D
:10215000E688F788D801ED91FC910484F585E02D9F
:1021600062E070E0C8010995482F60E070E0CE01A0
:10217000F7010995E881F981E688F788D801ED91A2
:10218000FC910484F585E02D6DE070E0C8010995AF
:10219000482F6DE070E0CE01F7010995E881F981E3
:1021A000E688F788D801ED91FC910484F585E02D4F
:1021B0006EE070E0C8010995482F6EE070E0CE0136
:1021C000F7010995E881F981E688F788D801ED9152
:1021D000FC910484F585E02D6BE070E0C801099561
:1021E000482F6BE070E0CE01F7010995E881F98195
:1021F000E688F788D801ED91FC910484F585E02DFF
:102200006AE070E0C8010995482F6AE070E0CE01ED
:10221000F7010995E881F981E688F788D801ED9101
:10222000FC910484F585E02D68E070E0C801099513
:10223000482F68E070E0CE01F7010995E881F98147
:10224000E688F788D801ED91FC910484F585E02DAE
:1022500069E070E0C8010995482F69E070E0CE019F
:10226000F701DF91CF911F910F91FF90EF900994AB
:10227000EF92FF920F931F93CF93DF938B01EA01AD
:10228000E881F981E284F384DB01ED91FC91008423
:10229000F185E02D61E070E0C8010995482F61E00B
:1022A00070E0CE01F7010995E881F981E484F584B5
:1022B000D801ED91FC910284F385E02D61E070E09E
:1022C000C8010995482F61E070E0CE01F70109953A
:1022D000E881F981E284F384D801ED91FC910084D6
:1022E000F185E02D62E070E0C8010995482F62E0B9
:1022F00070E0CE01F7010995E881F981E484F58465
:10230000D801ED91FC910284F385E02D62E070E04C
:10231000C8010995482F62E070E0CE01F7010995E8
:10232000E881F981E688F788D801ED91FC91048471
:10233000F585E02D64E070E0C8010995482F64E060
:1023400070E0CE01F7010995E881F981E688F78808
:10235000D801ED91FC910484F585E02D6CE070E0EE
:10236000C8010995482F6CE070E0CE01F70109958E
:10237000E881F981E688F788D801ED91FC91048421
:10238000F585E02D61E070E0C8010995482F61E016
:1023900070E0CE01F7010995E881F981E688F788B8
:1023A000D801ED91FC910484F585E02D62E070E0A8
:1023B000C8010995482F62E070E0CE01F701099548
:1023C000E881F981E688F788D801ED91FC910484D1
:1023D000F585E02D63E070E0C8010995482F63E0C2
:1023E00070E0CE01F7010995E881F981E688F78868
:1023F000D801ED91FC910484F585E02D60E070E05A
:10240000C8010995482F60E070E0CE01F7010995F9
:10241000E881F981E688F788D801ED91FC91048480
:10242000F585E02D6DE070E0C8010995482F6DE05D
:1024300070E0CE01F7010995E881F981E688F78817
:10244000D801ED91FC910484F585E02D6EE070E0FB
:10245000C8010995482F6EE070E0CE01F70109959B
:10246000E881F981E688F788D801ED91FC91048430
:10247000F585E02D6BE070E0C8010995482F6BE011
:1024800070E0CE01F7010995E881F981E688F788C7
:10249000D801ED91FC910484F585E02D6AE070E0AF
:1024A000C8010995482F6AE070E0CE01F70109954F
:1024B000E881F981E688F788D801ED91FC910484E0
:1024C000F585E02D68E070E0C8010995482F68E0C7
:1024D00070E0CE01F7010995E881F981E688F78877
:1024E000D801ED91FC910484F585E02D69E070E060
:1024F000C8010995482F69E070E0CE01F701DF912E
:10250000CF911F910F91FF90EF900994EF92FF925E
:102510000F931F93CF93DF938B01EA01E881F98139
:10252000E284F384DB01ED91FC910084F185E02DE0
:1025300060E070E0C8010995482F60E070E0CE01CE
:10254000F7010995E881F981E484F584D801ED91DA
:10255000FC910284F385E02D60E070E0C8010995EC
:10256000482F60E070E0CE01F701DF91CF911F911D
:102570000F91FF90EF9009944F925F926F927F922C
:10258000AF92BF92CF92DF92EF92FF920F931F9381
:10259000CF93DF93EB018A01DA01ED91FC91E284A4
:1025A000F384E881F9810084F185E02D61E070E039
:1025B000CE010995482F61E070E0C801F701099547
:1025C000D801ED91FC91E484F584E881F9810284DD
:1025D000F385E02D61E070E0CE010995482F61E0C0
:1025E00070E0C801F7010995E881F9810084F1855F
:1025F000E02D62E070E0CE010995682F880F770B1F
:1026000060587F4F072E000C880B990B0E94D72330
:1026100020E030E045E553E40E948C2420E030E0E7
:1026200044E752E40E942D236B017C01E881F9818B
:102630000284F385E02D62E070E0CE010995682FF9
:10264000880F770B60587F4F072E000C880B990B73
:102650000E94D72320E030E045E553E40E948C241B
:1026600020E030E044E752E40E942D232B013C019E
:10267000D801ED91FC91A284B38420E030E04FE7D3
:1026800053E4C701B6010E948724181664F020E0C5
:1026900030E040E053E4C701B6010E94BB220E9433
:1026A0009F23462F01C04FE762E070E0C801F501AB
:1026B0000995D801ED91FC91E484F58420E030E0A7
:1026C0004FE753E4C301B2010E948724181664F057
:1026D00020E030E040E053E4C301B2010E94BB229D
:1026E0000E949F23462F01C04FE762E070E0C801BF
:1026F000F7010995D801ED91FC91E688F788E8810A
:10270000F9810484F585E02D64E070E0CE0109953F
:10271000482F64E070E0C801F7010995D801ED91F8
:10272000FC91E688F788E881F9810484F585E02D3D
:102730006CE070E0CE010995482F6CE070E0C801B4
:10274000F7010995D801ED91FC91E688F788E881B9
:10275000F9810484F585E02D61E070E0CE010995F2
:10276000482F61E070E0C801F7010995D801ED91AB
:10277000FC91E688F788E881F9810484F585E02DED
:1027800062E070E0CE010995482F62E070E0C80178
:10279000F7010995D801ED91FC91E688F788E88169
:1027A000F9810484F585E02D63E070E0CE010995A0
:1027B000482F63E070E0C801F7010995D801ED9159
:1027C000FC91E688F788E881F9810484F585E02D9D
:1027D00060E070E0CE010995482F60E070E0C8012C
:1027E000F7010995D801ED91FC91E688F788E88119
:1027F000F9810284F385E02D62E070E0CE01099555
:10280000D82EE881F9810484F585E02D6DE070E033
:10281000CE01099541E0BDEBDB160CF440E0482BFE
:102820006DE070E0C801F7010995D801ED91FC91C8
:10283000E688F788E881F9810084F185E02D62E07F
:1028400070E0CE010995D82EE881F9810484F585E0
:10285000E02D6EE070E0CE01099541E0BDEBDB16A6
:102860000CF440E0482B6EE070E0C801F7010995D8
:10287000D801ED91FC91E688F788E881F98104841C
:10288000F585E02D6BE070E0CE010995482F6BE0F7
:1028900070E0C801F7010995D801ED91FC91E68837
:1028A000F788E881F9810484F585E02D6AE070E01D
:1028B000CE010995482F6AE070E0C801F70109953B
:1028C000D801ED91FC91E688F788E881F9810484CC
:1028D000F585E02D68E070E0CE010995482F68E0AD
:1028E00070E0C801F7010995D801ED91FC91E688E7
:1028F000F788E881F9810484F585E02D69E070E0CE
:10290000CE010995482F69E070E0C801F701DF9119
:10291000CF911F910F91FF90EF90DF90CF90BF90DC
:10292000AF907F906F905F904F9009940F931F939B
:10293000CF938C01C62F0E94A522C81721F06C2FBF
:10294000C8010E94AD228C2FCF911F910F91089545
:10295000CF92DF92FF920F931F93CF93DF938C015F
:10296000EA01E881F981C284D384DC011796ED91F4
:10297000FC91189782859385DC01ED91FC91019083
:10298000F081E02D0995F82ED8011796ED91FC9174
:10299000189780859185DC01ED91FC910190F08183
:1029A000E02D0995F69486954F2D481B61E070E067
:1029B000CE01F6010995E881F981C484D584D80156
:1029C0001796ED91FC91189786859785DC01ED911E
:1029D000FC910190F081E02D0995F82ED801179611
:1029E000ED91FC91189784859585DC01ED91FC9122
:1029F0000190F081E02D0995F69486954F2D481BA6
:102A000061E070E0CE01F6010995E881F981C284A8
:102A1000D384D8011796ED91FC91189780899189FC
:102A2000DC01ED91FC910190F081E02D0995482F9A
:102A300062E070E0CE01F6010995E881F981C48475
:102A4000D584D8011796ED91FC91189782899389C6
:102A5000DC01ED91FC910190F081E02D0995482F6A
:102A600062E070E0CE01F6010995E881F981C6883F
:102A7000D788D8011796ED91FC911897848995898C
:102A8000DC01ED91FC910280F381E02D099541E09C
:102A9000811101C040E060E070E0CE01F6010995CF
:102AA000E881F981C688D788D8011796ED91FC9105
:102AB000189786899789DC01ED91FC910280F3815A
:102AC000E02D099541E0811101C040E061E070E036
:102AD000CE01F6010995E881F981C688D788D80129
:102AE0001796ED91FC911897808D918DDC01ED91F9
:102AF000FC910280F381E02D099541E0811101C034
:102B000040E062E070E0CE01F6010995E881F981CC
:102B1000C688D788D8011796ED91FC911897828DB9
:102B2000938DDC01ED91FC910280F381E02D0995FC
:102B300041E0811101C040E063E070E0CE01F601A8
:102B40000995E881F981C688D788D8011796ED9153
:102B5000FC911897848D958DDC01ED91FC9102809C
:102B6000F381E02D099541E0811101C040E064E06E
:102B700070E0CE01F6010995E881F981C688D78811
:102B8000D8011796ED91FC911897868D978DDC01F1
:102B9000ED91FC910280F381E02D099541E08111D6
:102BA00001C040E068E070E0CE01F6010995E881DF
:102BB000F981C688D788D8011796ED91FC911897AE
:102BC00080A191A1DC01ED91FC910280F381E02DC7
:102BD000099541E0811101C040E069E070E0CE015B
:102BE000F6010995E881F981C688D788D80117963A
:102BF000ED91FC91189782A193A1DC01ED91FC91DC
:102C00000280F381E02D099541E0811101C040E08F
:102C10006AE070E0CE01F6010995E881F981C68885
:102C2000D788D8011796ED91FC91189784A195A1AA
:102C3000DC01ED91FC910280F381E02D099541E0EA
:102C4000811101C040E06BE070E0CE01F601099512
:102C5000E881F981C688D788D8011796ED91FC9153
:102C6000189786A197A1DC01ED91FC910280F38178
:102C7000E02D099541E0811101C040E06CE070E079
:102C8000CE01F6010995E881F981C688D788D80177
:102C90001796ED91FC91189780A591A5DC01ED9117
:102CA000FC910280F381E02D099541E0811101C082
:102CB00040E06DE070E0CE01F6010995E881F98110
:102CC000C688D788D8011796ED91FC91189782A5F0
:102CD00093A5DC01ED91FC910280F381E02D099533
:102CE00041E0811101C040E06EE070E0CE01F601EC
:102CF000DF91CF911F910F91FF90DF90CF900994BA
:102D0000CF93DF93FC018681A381B4816281882304
:102D100069F0062E000C770BED91FC91119706805F
:102D2000F781E02DCD01DF91CF910994EF01062EBF
:102D3000000C770BED91FC9111970680F781E02D47
:102D4000CD0109952FEF30E0A901481B51092D81D4
:102D500030E020583F4F81E0241735070CF480E025
:102D6000DF91CF9108958F929F92AF92BF92CF92B1
:102D7000DF92EF92FF92CF93DF93EC012E818B8154
:102D80009C816A81062E000C770BDC01ED91FC9191
:102D90000680F781E02D222311F0099502C00995E4
:102DA00080959D81E92EF12C282F30E0A701405815
:102DB0005F4F421753070CF04CC0682F691B6058D7
:102DC00070E080E090E00E94D5234B015C016FE74A
:102DD00070E06E197F09072E000C880B990B0E947A
:102DE000D7239B01AC01C501B4010E942D2320E033
:102DF00030E04FE753E40E948C246B017C0120E01B
:102E000030E0A9010E94282318161CF520E030E0CC
:102E10004FE753E4C701B6010E94872487FF1BC018
:102E200020E030E0A901C701B6010E94872420E01C
:102E300030E040E05FE387FD05C0C701B6010E94B6
:102E4000BC2204C0C701B6010E94BB220E949F237E
:102E500003C060E001C06FEF862FDF91CF91FF903C
:102E6000EF90DF90CF90BF90AF909F908F9008959C
:102E7000CF93DF93EC012E818B819C816A81062E9A
:102E8000000C770BDC01ED91FC910680F781E02DC1
:102E9000222331F009952FEF30E0281B310903C0C0
:102EA0000995282F30E04D8150E081E02417350747
:102EB0000CF480E0DF91CF9108958F929F92AF92B2
:102EC000BF92CF92DF92EF92FF92CF93DF93EC010C
:102ED0002E818B819C816A81062E000C770BDC0190
:102EE000ED91FC910680F781E02D222319F00995E0
:102EF000809501C00995682F880F770BED80F12C24
:102F00006E157F050CF44CC06E197F09072E000C5E
:102F1000880B990B0E94D7234B015C016FEF70E087
:102F20006E197F09072E000C880B990B0E94D7237E
:102F30009B01AC01C501B4010E942D2320E030E0CB
:102F40004FE753E40E948C246B017C0120E030E0C9
:102F5000A9010E94282318161CF520E030E04FE755
:102F600053E4C701B6010E94872487FF1BC020E0FD
:102F700030E0A901C701B6010E94872420E030E0BB
:102F800040E05FE387FD05C0C701B6010E94BC2297
:102F900004C0C701B6010E94BB220E949F2303C048
:102FA00060E001C06FEF862FDF91CF91FF90EF902F
:102FB000DF90CF90BF90AF909F908F900895CF9368
:102FC000DF93EC018B819C816A81062E000C770BCC
:102FD000DC01ED91FC910484F585E02D09958823B1
:102FE00011F08D8101C080E0DF91CF910895FC0147
:102FF000A381B4816281062E000C770BED91FC91C8
:1030000011970484F585E02DCD01099480E00895A1
:1030100020912D0330912E032115310529F0682FC1
:10302000C90101960C9496140895682F80912D0380
:1030300090912E03009711F00C94961408950F931D
:103040001F93CF93DF938C0185E791E0F801918383
:10305000808381E891E093838283C0E0D0E0F8012F
:103060002581368187819085C217D30764F49E013C
:10307000220F331FFC01E20FF31F808191810E9418
:10308000BF252196ECCF009731F0DF91CF911F91B2
:103090000F910C94BF25DF91CF911F910F9108954F
:1030A00080912D0390912E03892BF9F480E00E94EA
:1030B000F70890932E0380932D03892BB1F462E0DF
:1030C00070E080E00E946C0890932E0380932D03A3
:1030D000009759F061E00E94961480912D03909121
:1030E0002E0360E001960C94961408950F931F939D
:1030F000CF93DF938C01EB01FC018381E881F9819F
:10310000882359F00088F189E02DCB0109958823A7
:1031100009F4F6C0F8011382F3C00484F585E02DAC
:1031200064E070E0CE010995882381F083E090E0AF
:103130000E942725FC01128225EA31E03183208399
:10314000BC01CE010E942D0980E017C0E881F98101
:103150000484F585E02D61E070E0CE0109958823B7
:1031600091F081E190E00E9427258C010E940A1DC8
:10317000B801CE010E942D0981E0DF91CF911F910E
:103180000F910C941518E881F9810484F585E02DE0
:103190006EE070E0CE0109958823A9F082E090E00E
:1031A0000E9427252FE931E0FC0131832083BC01F7
:1031B000CE010E9448098E819F819B838A831F8252
:1031C0001E8280E097C0E881F9810484F585E02DB6
:1031D00063E070E0CE010995882369F088E190E012
:1031E0000E9427258C010E94B307B801CE010E94DE
:1031F0002D0982E0C2CFE881F9810484F585E02DB4
:1032000069E070E0CE0109958823A9F082E090E0A2
:103210000E94272529E931E0FC0131832083BC018C
:10322000CE010E9448098E819F819B838A831F82E1
:103230001E8281E05FC0E881F9810484F585E02D7C
:1032400068E070E0CE0109958823A9F082E090E063
:103250000E94272527E831E0FC0131832083BC014F
:10326000CE010E9448098E819F819B838A831F82A1
:103270001E8284E03FC0E881F9810484F585E02D59
:103280006AE070E0CE0109958823A9F082E090E021
:103290000E94272523E931E0FC0131832083BC0112
:1032A000CE010E9448098E819F819B838A831F8261
:1032B0001E8282E01FC0E881F9810484F585E02D3B
:1032C0006BE070E0CE0109958823D1F082E090E0B8
:1032D0000E9427252DE831E0FC0131832083BC01C9
:1032E000CE010E9448098E819F819B838A831F8221
:1032F0001E8283E0DF91CF911F910F910C940818EB
:10330000DF91CF911F910F910895EF92FF920F934C
:103310001F93CF93DF938B01EA01E881F981E28467
:10332000F384DB01ED91FC910084F185E02D61E0F7
:1033300070E0C8010995482F61E070E0CE01F70107
:103340000995E881F981E484F584D801ED91FC9137
:103350000284F385E02D61E070E0C8010995482FF3
:1033600061E070E0CE01F7010995E881F981E2841E
:10337000F384D801ED91FC910484F585E02D6EE095
:1033800070E0C8010995811102C042E801C04FE711
:1033900062E070E0CE01F7010995E881F981E484EB
:1033A000F584D801ED91FC910484F585E02D6DE064
:1033B00070E0C8010995811102C042E801C04FE7E1
:1033C00062E070E0CE01F7010995E881F981E688B5
:1033D000F788D801ED91FC910484F585E02D64E037
:1033E00070E0C8010995482F64E070E0CE01F70154
:1033F0000995E881F981E688F788D801ED91FC917B
:103400000484F585E02D6CE070E0C8010995482F33
:103410006CE070E0CE01F7010995E881F981E6885A
:10342000F788D801ED91FC910484F585E02D61E0E9
:1034300070E0C8010995482F61E070E0CE01F70106
:103440000995E881F981E688F788D801ED91FC912A
:103450000484F585E02D62E070E0C8010995482FED
:1034600062E070E0CE01F7010995E881F981E68814
:10347000F788D801ED91FC910484F585E02D63E097
:1034800070E0C8010995482F63E070E0CE01F701B4
:103490000995E881F981E688F788D801ED91FC91DA
:1034A0000484F585E02D60E070E0C8010995482F9F
:1034B00060E070E0CE01F7010995E881F981E688C6
:1034C000F788D801ED91FC910484F585E02D6DE03D
:1034D00070E0C8010995482F6DE070E0CE01F7015A
:1034E0000995E881F981E688F788D801ED91FC918A
:1034F0000484F585E02D6EE070E0C8010995482F41
:103500006EE070E0CE01F7010995E881F981E68867
:10351000F788D801ED91FC910484F585E02D6BE0EE
:1035200070E0C8010995482F6BE070E0CE01F7010B
:103530000995E881F981E688F788D801ED91FC9139
:103540000484F585E02D6AE070E0C8010995482FF4
:103550006AE070E0CE01F7010995E881F981E6881B
:10356000F788D801ED91FC910484F585E02D68E0A1
:1035700070E0C8010995482F68E070E0CE01F701BE
:103580000995E881F981E688F788D801ED91FC91E9
:103590000484F585E02D69E070E0C8010995482FA5
:1035A00069E070E0CE01F701DF91CF911F910F919B
:1035B000FF90EF900994DF92EF92FF920F931F9389
:1035C000CF93DF93EC018B017A018C819D81813057
:1035D000910521F0029709F471C011C0DB01ED9152
:1035E000FC910288F389E02DCB010995882329F00D
:1035F00082E090E09D838C83DDC11D821C82D80116
:10360000ED91FC910084F185E02D60E070E0C8014F
:103610000995D801ED91FC910284F385E02D60E0DD
:1036200070E0C8010995D801ED91FC910084F18505
:10363000E02D60E070E0C8010995682F880F770BD6
:10364000880B990B0E94D723AB01BC01CE010E94CD
:10365000A909D82ED801ED91FC910284F385E02DC3
:1036600060E070E0C8010995682F880F770B880B20
:10367000990B0E94D723AB01BC01CE010E94A9097E
:10368000C82FD701ED91FC910284F385E02D4D2DDB
:1036900060E070E0C7010995D701ED91FC910484C9
:1036A000F585E02D4C2F60E070E0C701DF91CF91F0
:1036B0001F910F91FF90EF90DF900994AF81B88533
:1036C000A750BE4FFA0180819181FC01228533858C
:1036D0004C9160E070E0C701F9010995A985BA85B0
:1036E000A750BE4FF70180819181FC01248535856B
:1036F0004C9160E070E0C701F9010995D801ED91A6
:10370000FC910288F389E02DC8010995882309F40A
:1037100054C18E81D801ED91FC910484F585E02D92
:10372000882309F468C062E070E0C801099581113E
:103730005FC1D801ED91FC910484F585E02D63E033
:1037400070E0C8010995811153C1D801ED91FC9138
:103750000484F585E02D61E070E0C80109958111D0
:1037600047C1D801ED91FC910484F585E02D60E01E
:1037700070E0C801099581113BC1D801ED91FC9120
:103780000484F585E02D68E070E0C8010995811199
:103790002FC1D801ED91FC910484F585E02D69E0FD
:1037A00070E0C8010995811123C1D801ED91FC9108
:1037B0000484F585E02D6AE070E0C8010995811167
:1037C00017C1D801ED91FC910484F585E02D6CE0E2
:1037D00070E0C801099581110BC1D801ED91FC91F0
:1037E0000484F585E02D64E070E0C801099581113D
:1037F000FFC01E82FDC063E070E0C8010995882308
:1038000051F08F8198858230910514F0019719C08D
:1038100081E090E016C0D801ED91FC910484F5851B
:10382000E02D62E070E0C8010995882369F02F81DE
:10383000388589859A8501972817390714F4C901B5
:10384000019698878F83B6C0D801ED91FC910484CE
:10385000F585E02D61E070E0C8010995882361F0ED
:1038600029853A858F8198850196821793070CF0F8
:1038700051C0C90101974EC0D801ED91FC9104845B
:10388000F585E02D60E070E0C8010995882351F0CE
:1038900089859A858E37910514F401963BC08EE791
:1038A00090E038C0D801ED91FC910484F585E02DBD
:1038B00064E070E0C80109958823D1F08B818130E4
:1038C00049F0823071F087E190E098878F8385E23C
:1038D00090E020C084E190E098878F8380E290E0C0
:1038E00019C08EE190E098878F8389E290E012C042
:1038F000D801ED91FC910484F585E02D6CE070E039
:10390000C8010995882349F088E090E098878F8363
:103910008AE290E09A8789874DC0D801ED91FC91A9
:103920000484F585E02D68E070E0C80109958823DE
:1039300069F082E08B838EE190E09E878D8789E23B
:1039400090E09C878B8789E490E032C0D801ED91AC
:10395000FC910484F585E02D6AE070E0C8010995CA
:10396000882379F081E08B8324E130E03E872D8746
:1039700020E230E03C872B8725E330E0388B2F872F
:103980001AC0D801ED91FC910484F585E02D69E021
:1039900070E0C8010995882359F11B8287E190E006
:1039A0009E878D8785E290E09C878B8787E490E0F7
:1039B000988B8F8781E08E831BC080912B03909121
:1039C0002C03009799F06F810E94961480912B032D
:1039D00090912C03698501960E94961480912B0387
:1039E00090912C036B8102960E9496141D821C827A
:1039F000DF91CF911F910F91FF90EF90DF9008958D
:103A0000CF93DF93EC010E941F18CE01DF91CF917D
:103A10000C94BF250F931F93CF93DF93EC011A8271
:103A200087EF91E0998388831B8200912B0310918B
:103A30002C0301151105F1F581E00E94F7088C01B6
:103A400090932C0380932B03892BA1F563E070E006
:103A500081E00E946C0890932C0380932B031B82BF
:103A600027E130E03E872D8725E230E03C872B8739
:103A700027E430E0388B2F8728E030E038872F8329
:103A80002AE230E03A872987009731F168E00E9406
:103A9000961480912B0390912C03698501960E94C6
:103AA000961480912B0390912C036B8102960E94B7
:103AB000961412C0C8010E94A52290E098878F83B7
:103AC000C80101960E94A52290E09A878987C801C3
:103AD00002960E94A5228B838B81813069F082300F
:103AE000B1F087E190E09E878D8785E290E09C872A
:103AF0008B8787E490E015C084E190E09E878D87F6
:103B000080E290E09C878B8785E390E00AC08EE19D
:103B100090E09E878D8789E290E09C878B8789E47F
:103B200090E0988B8F8789859A858038910524F05D
:103B30008EE790E09A87898789859A852F813885D5
:103B4000821793071CF4019798878F8381E090E098
:103B50009D838C83DF91CF911F910F910895CF9317
:103B6000DF9300D01F92CDB7DEB7789484B5826022
:103B700084BD84B5816084BD85B5826085BD85B511
:103B8000816085BD80916E00816080936E0010928F
:103B9000810080918100826080938100809181000A
:103BA000816080938100809180008160809380009B
:103BB0008091B10084608093B1008091B0008160F9
:103BC0008093B00080917A00846080937A00809125
:103BD0007A00826080937A0080917A00816080937D
:103BE0007A0080917A00806880937A001092C100F8
:103BF000E0919C02F0919D0282E08083E091980226
:103C0000F09199021082E0919A02F0919B0280E17A
:103C100080831092A402E091A002F091A10286E0BC
:103C20008083E0919E02F0919F0280818061808379
:103C3000E0919E02F0919F02808188608083E091F4
:103C40009E02F0919F02808180688083E0919E02B5
:103C5000F0919F0280818F7D8083809100019091FF
:103C600001010197909301018093000143E050E02E
:103C700062E070E0CE0101960E9495228981853A2A
:103C800031F48A818E3919F48B818C3811F080E0FF
:103C90004DC089E090E00E94A5228233A1F162E349
:103CA00089E090E00E94961410928B0210928A0292
:103CB00060E080E090E00E94961460918A0281E0CA
:103CC00090E00E9496148091180190911901A091A2
:103CD0001A0189839A83AB83CE0101967C0102E0AD
:103CE00010E0D701DD907D01C8010E94A522D81601
:103CF00021F06D2DC8010E94AD220F5F1F4F0530CE
:103D0000110579F712C080E090E00E94A52290E0B2
:103D100090938B0280938A0281E090E00E94A5221A
:103D200090E090938B0280938A0281E080937E02E0
:103D30008BE491E00E9427257C018FE191E0F7015F
:103D400091838083339681E2DF011D928A95E9F7A2
:103D5000EB5BFE4F83E0DF011D928A95E9F7F701E7
:103D600014A6F0927D02E0927C028CEB90E00E941F
:103D700027258C018DE591E0D80111969C938E93B7
:103D8000C8018E589F4F1D969C938E931C9780E47C
:103D900090E01B969C938E931A971E961C921E97EA
:103DA00091961C9291978AE0EFE4F1E0579601908A
:103DB0000D928A95E1F710937B0200937A0283E0DB
:103DC0000E942B0E83E00E94030EF701128289E00D
:103DD00090E00E9427257C01DC0114961C92149728
:103DE00085E791E011969C938E9381E891E013967C
:103DF0009C938E93129786E190E016969C938E93F7
:103E000015978CE290E00E9427256C01F7019087BE
:103E1000878321E040E063E0C8010E945B09D6018E
:103E20008D939C93F701C780D08420E040E063E04D
:103E3000C8010E945B09D60113969C938E9312973A
:103E4000F701C780D08421E041E063E0C8010E940F
:103E50005B09D60115969C938E931497F701C78042
:103E6000D08420E041E063E0C8010E945B09D601F4
:103E700017969C938E931697F701C780D08421E004
:103E800042E063E0C8010E945B09D60119969C9349
:103E90008E931897F701C780D08420E042E063E05A
:103EA000C8010E945B09D6011B969C938E931A97BA
:103EB000F701C780D08421E043E063E0C8010E949D
:103EC0005B09D6011D969C938E931C97F701C780C2
:103ED000D08420E043E063E0C8010E945B09D60182
:103EE0001F969C938E931E97F701C780D08421E084
:103EF00044E062E0C8010E945B09D60151969C93A0
:103F00008E935097F701C780D08421E045E062E0AE
:103F1000C8010E945B09D60153969C938E935297D9
:103F2000F701C780D08420E040E061E0C8010E9432
:103F30005B09D60155969C938E935497F701C780E1
:103F4000D08420E041E061E0C8010E945B09D60115
:103F500057969C938E935697F701C780D08420E0A4
:103F600042E061E0C8010E945B09D60159969C932A
:103F70008E935897F701C780D08420E043E061E03A
:103F8000C8010E945B09D6015B969C938E935A9759
:103F9000F701C780D08420E044E061E0C8010E94BE
:103FA0005B09D6015D969C938E935C97F701C78061
:103FB000D08420E048E061E0C8010E945B09D6019E
:103FC0005F969C938E935E97F701C780D08420E024
:103FD00049E061E0C8010E945B09D60191969C937B
:103FE0008E939097F701C780D08420E04AE061E08B
:103FF000C8010E945B09D60193969C938E93929779
:10400000F701C780D08420E04BE061E0C8010E9446
:104010005B09D60195969C938E939497F701C78080
:10402000D08420E04CE061E0C8010E945B09D60129
:1040300097969C938E939697F701C780D08420E043
:104040004DE061E0C8010E945B09D60199969C93FE
:104050008E939897F701E780F08420E04EE061E0CE
:10406000C8010E945B09D7019B969C938E939A97F7
:104070000E94501880912D0390912E03009769F0B3
:1040800001960E94A5228230B1F018F4813061F0CF
:1040900004C08330B9F08430F9F082E090E00E94EF
:1040A00027252FE931E01EC082E090E00E942725FD
:1040B00029E931E00DC082E090E00E94272523E944
:1040C00031E010C082E090E00E9427252DE831E029
:1040D000DC012D933C9309C082E090E00E942725EB
:1040E00027E831E0FC01318320836C010E945018E5
:1040F00080912D0390912E03009731F00E94A5220C
:10410000813081F08230B1F083E090E00E94272579
:10411000DC0112961C92129725EA31E02D933C9314
:104120008C010FC081E190E00E9427258C010E9444
:104130000A1D07C088E190E00E9427258C010E949B
:10414000B307A0907C02B0907D02E0907A02F090DC
:104150007B0285E00E942B0E85E00E94030E84E026
:104160000E942B0E84E00E94030EF701B186A08608
:1041700002831383C482D582178216823BEA632EA0
:1041800031E0732E5524539448E0242E312C809135
:104190007E02882309F41CC180917C0290917D02EB
:1041A000DC01ED91FC910190F081E02D09958111E8
:1041B000F7C000917A0210917B02F8018685C484D1
:1041C000D584A284B384882351F1E12CF12CEA1424
:1041D000FB0464F5C701F7FC079623E095958795E6
:1041E0002A95E1F7F601E80FF91F2081022E000C55
:1041F000330BC701B1010E94F92402C03595279500
:104200008A95E2F7C9018170992720FF02C081E3F6
:1042100090E00E94720EFFEFEF1AFF0AD8CF7601EE
:10422000C7018C199D098A159B057CF08AE090E0F6
:104230000E94720ED801ED91FC910684F785E02D65
:10424000C801099581110EC038C0F70181917F0125
:10425000882319F081E390E002C080E090E00E94A2
:10426000720EDECFD8011296ED91FC911397309724
:1042700019F08281811121C084E090E00E942725FD
:104280007C01FC017182608253825282892B09F485
:10429000A2C0F80186819781009711F00E94BF2586
:1042A000D80112968D919C91139717969C938E939B
:1042B00016971396FC92EE921297C0900001D09040
:1042C00001010D2C000CEE08FF080E94770E4B0137
:1042D0005C01C114D104E104F104F1F00E94770EF5
:1042E000DC01CB0188199909AA09BB09883E9340D2
:1042F000A105B10570F3F1E0CF1AD108E108F1088A
:1043000028EE820E23E0921EA11CB11CC114D10420
:10431000E104F10419F7DDCFF89400917A021091CD
:104320007B02D801ED91FC910480F581E02DC8015C
:104330000995F80180859185DC01ED91FC9100845F
:10434000F185E02D0995F80182819381009751F064
:1043500040855185DC01ED91FC910190F081E02DCB
:10436000B8010995F80186819781892B71F48481C0
:104370009581009751F040855185DC01ED91FC91CC
:104380000190F081E02DB801099580917C02909117
:104390007D02DC01ED91FC910480F581E02D099511
:1043A00080917C0290917D02DC01ED91FC91028074
:1043B000F381E02D0995F89480917C0290917D0223
:1043C000DC01ED91FC910680F781E02D0995789450
:1043D0000E94ED01DCCEF801868197819383828370
:1043E000178216826ACFECE8F2E01382128288EE1E
:1043F00093E0A0E0B0E084839583A683B78385EE45
:1044000091E09183808385EC90E09587848784ECAC
:1044100090E09787868780EC90E0918B808B81EC91
:1044200090E0938B828B82EC90E0958B848B86EC72
:1044300090E0978B868B118E128E138E148E1092B5
:104440002A031092290310922C0310922B0310922E
:104450002E0310922D030895CF92DF92EF92FF92D8
:104460000F931F93CF937C018A01DA01ED91FC91A8
:10447000C284D384DC011796ED91FC911897828158
:104480009381DC01ED91FC910190F081E02D099583
:10449000C82FD7011796ED91FC91189780819181D3
:1044A000DC01ED91FC910190F081E02D0995C6951C
:1044B00086954C2F481B60E070E0C801F601099515
:1044C000D801ED91FC91C484D584D7011796ED9164
:1044D000FC91189786819781DC01ED91FC91019008
:1044E000F081E02D0995C82FD7011796ED91FC9129
:1044F000189784819581DC01ED91FC910190F08108
:10450000E02D0995C69586954C2F481B60E070E01C
:10451000C801F601CF911F910F91FF90EF90DF90AE
:10452000CF90099402970C942C22DC01CB01FC0162
:10453000F999FECF06C0F2BDE1BDF89A319600B4FC
:104540000D9241505040B8F70895F999FECF92BDB1
:1045500081BDF89A992780B50895262FF999FECF45
:104560001FBA92BD81BD20BD0FB6F894FA9AF99A90
:104570000FBE019608955058BB27AA270E94D32248
:104580000C944D240E943F2438F00E94462420F0D1
:1045900039F49F3F19F426F40C943C240EF4E09572
:1045A000E7FB0C943624E92F0E945E2458F3BA17D7
:1045B000620773078407950720F079F4A6F50C9439
:1045C00080240EF4E0950B2EBA2FA02D0B01B9011B
:1045D00090010C01CA01A0011124FF27591B99F079
:1045E000593F50F4503E68F11A16F040A22F232F85
:1045F000342F4427585FF3CF469537952795A795D5
:10460000F0405395C9F77EF41F16BA0B620B730B7B
:10461000840BBAF09150A1F0FF0FBB1F661F771FEC
:10462000881FC2F70EC0BA0F621F731F841F48F4A1
:10463000879577956795B795F7959E3F08F0B0CF2A
:104640009395880F08F09927EE0F97958795089511
:104650000E94122408F481E008950E9441230C94E2
:104660004D240E94462458F00E943F2440F029F433
:104670005F3F29F00C94362451110C9481240C9442
:104680003C240E945E2468F39923B1F3552391F3EF
:10469000951B550BBB27AA2762177307840738F0B1
:1046A0009F5F5F4F220F331F441FAA1FA9F335D00E
:1046B0000E2E3AF0E0E832D091505040E695001CC2
:1046C000CAF72BD0FE2F29D0660F771F881FBB1F7C
:1046D000261737074807AB07B0E809F0BB0B802D5A
:1046E000BF01FF2793585F4F3AF09E3F510578F086
:1046F0000C9436240C9481245F3FE4F3983ED4F369
:10470000869577956795B795F7959F5FC9F7880F59
:10471000911D9695879597F90895E1E0660F771FAB
:10472000881FBB1F621773078407BA0720F0621B3C
:10473000730B840BBA0BEE1F88F7E09508950E9467
:10474000A6236894B1110C94812408950E946624D4
:1047500088F09F5798F0B92F9927B751B0F0E1F042
:10476000660F771F881F991F1AF0BA95C9F714C0F2
:10477000B13091F00E948024B1E008950C9480241F
:10478000672F782F8827B85F39F0B93FCCF386952B
:1047900077956795B395D9F73EF490958095709588
:1047A00061957F4F8F4F9F4F0895E89409C097FB05
:1047B0003EF490958095709561957F4F8F4F9F4FF8
:1047C0009923A9F0F92F96E9BB279395F69587953C
:1047D00077956795B795F111F8CFFAF4BB0F11F4FF
:1047E00060FF1BC06F5F7F4F8F4F9F4F16C08823A6
:1047F00011F096E911C0772321F09EE8872F762FDC
:1048000005C0662371F096E8862F70E060E02AF01C
:104810009A95660F771F881FDAF7880F9695879508
:1048200097F90895990F0008550FAA0BE0E8FEEFDD
:1048300016161706E807F907C0F012161306E40764
:10484000F50798F0621B730B840B950B39F40A265D
:1048500061F0232B242B252B21F408950A2609F43B
:10486000A140A6958FEF811D811D089597F99F673F
:1048700080E870E060E008959FEF80EC08950024E8
:104880000A941616170618060906089500240A94B5
:1048900012161306140605060895092E0394000C3B
:1048A00011F4882352F0BB0F40F4BF2B11F460FFCA
:1048B00004C06F5F7F4F8F4F9F4F089557FD9058F3
:1048C000440F551F59F05F3F71F04795880F97FBD4
:1048D000991F61F09F3F79F087950895121613068E
:1048E0001406551FF2CF4695F1DF08C016161706BD
:1048F0001806991FF1CF86957105610508940895F2
:10490000E894BB2766277727CB0197F908950E9483
:10491000122408F48FEF08950E949F240C944D24D4
:104920000E943F2438F00E94462420F0952311F085
:104930000C9436240C943C2411240C9481240E9461
:104940005E2470F3959FC1F3950F50E0551F629F51
:10495000F001729FBB27F00DB11D639FAA27F00DD8
:10496000B11DAA1F649F6627B00DA11D661F829FFF
:104970002227B00DA11D621F739FB00DA11D621FE4
:10498000839FA00D611D221F749F3327A00D611D01
:10499000231F849F600D211D822F762F6A2F1124E3
:1049A0009F5750409AF0F1F088234AF0EE0FFF1F16
:1049B000BB1F661F771F881F91505040A9F79E3F6D
:1049C000510580F00C9436240C9481245F3FE4F36D
:1049D000983ED4F3869577956795B795F795E795C3
:1049E0009F5FC1F7FE2B880F911D9695879597F9CC
:1049F000089597FB072E16F4009407D077FD09D091
:104A00000E940D2507FC05D03EF4909581959F4F9F
:104A10000895709561957F4F0895AA1BBB1B51E1C6
:104A200007C0AA1FBB1FA617B70710F0A61BB70B1E
:104A3000881F991F5A95A9F780959095BC01CD01C3
:104A40000895EE0FFF1F0590F491E02D09940F9348
:104A50001F93CF93DF938230910510F482E090E0B2
:104A6000E0913103F091320320E030E0A0E0B0E0CB
:104A7000309719F1408151810281138148175907FC
:104A8000C8F08417950769F4109731F012960C93CB
:104A9000129713961C9327C000933103109332038F
:104AA00022C02115310519F04217530718F49A0155
:104AB000BD01EF01DF01F801DBCF21153105F9F070
:104AC000281B390B2430310580F48A819B816115C4
:104AD000710521F0FB019383828304C0909332031C
:104AE00080933103FE01329644C0FE01E20FF31FB2
:104AF0008193919322503109398328833AC02091C0
:104B00002F0330913003232B41F420911401309175
:104B100015013093300320932F032091120130911F
:104B200013012115310541F42DB73EB7409116010F
:104B300050911701241B350BE0912F03F0913003A6
:104B4000E217F307A0F42E1B3F0B2817390778F064
:104B5000AC014E5F5F4F2417350748F04E0F5F1FC3
:104B60005093300340932F038193919302C0E0E070
:104B7000F0E0CF01DF91CF911F910F910895CF9376
:104B8000DF93009709F481C0FC01329713821282EF
:104B9000A0913103B0913203109781F420813181CB
:104BA000820F931F20912F0330913003281739076C
:104BB00051F5F0933003E0932F0367C0ED0120E03F
:104BC00030E0CE17DF0740F44A815B819E0141153A
:104BD0005105F1F0EA01F5CFD383C28340815181C1
:104BE000840F951FC817D90759F488819981840FBC
:104BF000951F0296918380838A819B819383828310
:104C00002115310529F4F0933203E09331033DC0BF
:104C1000E901FB83EA8349915991C40FD51FEC1731
:104C2000FD0761F480819181840F951F0296E9014F
:104C300099838883828193819B838A83E0E0F0E07B
:104C400012968D919C911397009719F0FD01DC014C
:104C5000F7CF8D919C9111979D012E5F3F4F820F51
:104C6000931F20912F03309130032817390769F4DF
:104C7000309729F4109232031092310302C013824C
:104C80001282B0933003A0932F03DF91CF91089548
:104C900081E090E0F8940C945426DC0101C06D93FF
:0C4CA00041505040E0F70895F894FFCF19
:104CAC000C0009000300000000000101400300405B
:104CBC000301000033038000A59E8C000000004B14
:104CCC00024802D406D806C402BA02B202A4029860
:104CDC000254024E0259020000000000000000B510
:104CEC0000B500B500B500B500B500B500B50000C5
:104CFC00808080808000000202000000006B08D2DF
:104D0C0006110543023B02330216020A020002F7A7
:104D1C000100000000A8142C221F18001DFEFF002B
:104D2C00009222000000008519000000009C0E007B
:104D3C00000000EA0F00000000BC12000000003868
:104D4C001100000000861200000000761800000020
:104D5C0000B50000807F7F7F7F000000000000CF47
:104D6C0002000000005D17381700000000B3168029
:104D7C001600000000F717DF1700000000061806E9
:104D8C001800000000C1008700B0019107E101BFCD
:104D9C0001D30100000000DB1A00101112131415CE
:104DAC0016171718191A1B1B1C1D1E1E1F2021223B
:104DBC0022232424252626272828292A2A2B2C2C72
:104DCC002D2D2E2F2F3030313132333334343535C5
:104DDC003636373738383839393A3A3B3B3B3C3C36
:104DEC003D3D3D3E3E3F3F3F4040404041414142C2
:104DFC00424243434343434444444444454545456C
:104E0C004546464646464646464646474747474732
:0A4E1C00474747474747474747000D
:00000001FF
